:020000040800F2
:1000000000070020E50400089515000815150008F4
:100010006D1500081515000841150008E7040008D3
:10002000E7040008E7040008E7040008F9360008C0
:10003000E7040008E7040008E7040008E7040008F4
:10004000E7040008E7040008E7040008E7040008E4
:10005000E7040008E7040008253B0008513B0008BE
:100060007D3B0008A93B0008D53B0008E7040008D9
:10007000E7040008E7040008E7040008E7040008B4
:10008000E7040008E7040008E7040008AD240008BE
:10009000192500086D250008C1250008013C00084D
:1000A000E7040008E7040008E7040008E704000884
:1000B00075390008E7040008E7040008E7040008B1
:1000C000E7040008E7040008E7040008E704000864
:1000D000E70400086529000879290008E7040008FA
:1000E000693C0008E7040008E7040008E70400088A
:1000F000E7040008E7040008E7040008E704000834
:10010000E7040008E7040008E7040008E704000823
:10011000E7040008E7040008E7040008E704000813
:10012000E7040008E7040008E7040008E704000803
:10013000E7040008E7040008E7040008E7040008F3
:10014000E7040008E7040008E7040008E7040008E3
:10015000E7040008E7040008E7040008E7040008D3
:10016000E7040008E7040008E7040008E7040008C3
:10017000E7040008E7040008E7040008E7040008B3
:10018000E7040008E7040008E7040008E7040008A3
:10019000E7040008E7040008E7040008E704000893
:1001A000E7040008E7040008E7040008E704000883
:1001B000E7040008E7040008E7040008E704000873
:1001C000E7040008E7040008E7040008E704000863
:1001D000E7040008E7040008E7040008E704000853
:1001E00053B94AB9002908BF00281CBF4FF0FF319E
:1001F0004FF0FF3000F074B9ADF1080C6DE904CE9A
:1002000000F006F8DDF804E0DDE9022304B07047F1
:100210002DE9F047089D04468E46002B4DD18A42B9
:10022000944669D9B2FA82F252B101FA02F3C2F1EC
:10023000200120FA01F10CFA02FC41EA030E94407D
:100240004FEA1C48210CBEFBF8F61FFA8CF708FB9E
:1002500016E341EA034306FB07F199420AD91CEB76
:10026000030306F1FF3080F01F81994240F21C81A8
:10027000023E63445B1AA4B2B3FBF8F008FB1033F0
:1002800044EA034400FB07F7A7420AD91CEB040425
:1002900000F1FF3380F00A81A74240F207816444F5
:1002A000023840EA0640E41B00261DB1D44000237A
:1002B000C5E900433146BDE8F0878B4209D9002DDE
:1002C00000F0EF800026C5E9000130463146BDE868
:1002D000F087B3FA83F6002E4AD18B4202D38242D2
:1002E00000F2F980841A61EB030301209E46002D81
:1002F000E0D0C5E9004EDDE702B9FFDEB2FA82F2D6
:10030000002A40F09280A1EB0C014FEA1C471FFA33
:100310008CFE0126200CB1FBF7F307FB131140EA1A
:1003200001410EFB03F0884208D91CEB010103F1E7
:10033000FF3802D2884200F2CB804346091AA4B2A9
:10034000B1FBF7F007FB101144EA01440EFB00FE7D
:10035000A64508D91CEB040400F1FF3102D2A645E2
:1003600000F2BB800846A4EB0E0440EA03409CE781
:10037000C6F12007B34022FA07FC4CEA030C20FA2E
:1003800007F401FA06F31C43F9404FEA1C4900FA4E
:1003900006F3B1FBF9F8200C1FFA8CFE09FB1811CB
:1003A00040EA014108FB0EF0884202FA06F20BD93E
:1003B0001CEB010108F1FF3A80F08880884240F28E
:1003C0008580A8F102086144091AA4B2B1FBF9F0D2
:1003D00009FB101144EA014100FB0EFE8E4508D9CD
:1003E0001CEB010100F1FF346CD28E456AD9023852
:1003F000614440EA0840A0FB0294A1EB0E01A14237
:10040000C846A64656D353D05DB1B3EB080261EBA4
:100410000E0101FA07F722FA06F3F1401F43C5E97E
:10042000007100263146BDE8F087C2F12003D840B4
:100430000CFA02FC21FA03F3914001434FEA1C47F6
:100440001FFA8CFEB3FBF7F007FB10360B0C43EAE8
:10045000064300FB0EF69E4204FA02F408D91CEB98
:10046000030300F1FF382FD29E422DD90238634496
:100470009B1B89B2B3FBF7F607FB163341EA034136
:1004800006FB0EF38B4208D91CEB010106F1FF3885
:1004900016D28B4214D9023E6144C91A46EA00467C
:1004A00038E72E46284605E70646E3E61846F8E60E
:1004B0004B45A9D2B9EB020864EB0C0E0138A3E757
:1004C0004646EAE7204694E74046D1E7D0467BE738
:1004D000023B614432E7304609E76444023842E7B0
:1004E000704700BF02E000F000F8FEE772B63A483D
:1004F00080F30888394880F3098839484EF6085156
:10050000CEF20001086040F20000CCF200004EF68E
:100510003471CEF200010860BFF34F8FBFF36F8FCD
:1005200040F20000C0F2F0004EF68851CEF2000119
:100530000860BFF34F8FBFF36F8F4FF00000E1EE05
:10054000100A4EF63C71CEF200010860062080F3DE
:100550001488BFF36F8F03F04FF903F02BF903F00A
:1005600075F94FF055301F491B4A91423CBF41F885
:10057000040BFAE71C49194A91423CBF41F8040BAD
:10058000FAE71A491A4A1B4B9A423EBF51F8040B2C
:1005900042F8040BF8E700201749184A91423CBF83
:1005A00041F8040BFAE703F009F903F09DF9144C44
:1005B000144DAC4203DA54F8041B8847F9E700F005
:1005C00041F8114C114DAC4203DA54F8041B884732
:1005D000F9E703F0F1B80000000700200023002035
:1005E000000000080001002000070020F03F000884
:1005F000002300202423002028230020083C002082
:10060000E0010008E0010008E0010008E001000846
:100610002DE9F04F2DED108AC1F80CD0C3689D462E
:10062000BDEC108ABDE8F08F002383F311882846C3
:10063000A047002002F04CFDFEE702F0D1FC00DFF5
:10064000FEE700002DE9F04102F0F4FF074603F059
:100650003FF80546C0BB284B9F4235D001339F422F
:1006600035D0264B27F0FF029A4234D1F8B200F081
:100670004DFAA84642F2107400F052FC08B1002472
:10068000A04600F049FA064648B354BB464635B189
:100690001B4B9F4203D003F013F800242646002092
:1006A00002F0D2FF0EB100F02DF800F097FC00F040
:1006B00077FE00F071FF0546B4B900F041FD4FF43C
:1006C0007A7002F00BFDF7E7A8460024D4E7044651
:1006D0004FF00108D0E780464FF47A74CCE7044627
:1006E000D5E74FF47A74D2E700F056FF431BA342DC
:1006F000E3D900F007F8DCE7010007B0000008B01C
:10070000263A09B01E4B1F4A10B51C461968013124
:1007100034D004339342F9D162681B4B9A422DD9ED
:100720001A4B9B6803F1006303F580339A4225D28C
:1007300002F09AFF02F0ACFF002000F04BFE144BD9
:100740000220187000F082FE124B1A6C00221A640C
:10075000196E1A66196E596C5A64596E5A665B6E38
:1007600072B64FF0E0232021C3F8084DD4E90032DF
:1007700081F311889D4683F30888104710BD00BFA0
:100780000000010820000108FFFF000800230020EE
:100790002823002000380240094A136849F2690002
:1007A00099B21B0C00FB01331360064B186844F22E
:1007B000506182B2000C01FB0200186080B27047E9
:1007C000202300201C23002010B500211022044605
:1007D00000F050FE034B03CB206061601868A060FE
:1007E00010BD00BF107AFF1F2DE9F043224DBBB0B2
:1007F00000F0D2FEAB6840F2ED22C31A934232D928
:1008000006AFA8602B4628220021384601F08EFB57
:1008100005F10E0000F026FE002604465FFA80F97E
:1008200005F10E08F3B2F100994501F1280107D94D
:1008300008EB06030822384601F078FB0136F1E7A1
:1008400008230122CDE9023205340C4B0193A4B2F6
:1008500030230093CDE9047405A3D3E90023297B59
:10086000074801F07BF93BB0BDE8F083AFF30080AF
:1008700078F6339F93CACD8D6833002075330020FE
:100880004433002070B50D4614461E4601F0FCF8B6
:1008900050B9022E10D1012C0ED112A3D3E900239E
:1008A000C5E90023012007E0282C10D005D8012C31
:1008B00009D0052C0FD0002070BD302CFBD10BA32C
:1008C000D3E90023ECE70BA3D3E90023E8E70BA36C
:1008D000D3E90023E4E70BA3D3E90023E0E700BF5B
:1008E000AFF30080401DA12026812A0B78F6339FAC
:1008F00093CACD8D9E6AC421818A46EE26417272CA
:10090000DF25D7B7F017304A39059E5613B5044690
:100910002346084620220021019001F007FB22799E
:100920000198032A234628BF032203F8042F20211D
:10093000022201F0FBFA62790198072A234628BFB8
:10094000072203F8052F2221032201F0EFFAA279F2
:100950000198072A234628BF072203F8062F2521DE
:10096000032201F0E3FA019804F108031022282180
:1009700001F0DCFA382002B010BD00002DE9F04F84
:10098000ADF5017D21AD0EAE40F2751280460F46E9
:1009900022A80021296000F06DFD48220021304688
:1009A00000F068FD00F0F8FD564B4FF47A72B0FB92
:1009B000F2F0186093E80700012386E807000DF1C4
:1009C0005A003382FFF700FF40F60423338407AB5D
:1009D00018464D4903F0F2F9182230642946304692
:1009E00086F83C20FFF792FF12AB0446014608222E
:1009F000284601F09BFA0822A1180DF14903284668
:100A000001F094FA0DF14A03082204F1100128467E
:100A100001F08CFA13AB202204F11801284601F0F2
:100A200085FA14AB402204F13801284601F07EFA21
:100A300016AB082204F17801284601F077FA0DF18F
:100A40005903082204F18001284601F06FFA04F1ED
:100A5000880A0DF15A0904F5847B4B465146082259
:100A600028460AF1080A01F061FAD34509F10109A3
:100A7000F3D11BAB08225946284601F057FA04F57A
:100A800088744FF0000996F834304B450AD9B36B9F
:100A900021464B440822284601F048FA083409F15F
:100AA0000109F0E74FF0000996F83C304B4504EBA4
:100AB000C90108D9336C08224B44284601F036FAA4
:100AC00009F10109F0E700230393BB7E029307318C
:100AD00007F119030193C1F3CF010123CDE90451BB
:100AE0000093F97E05A3D3E90023404601F036F8D0
:100AF0000DF5017DBDE8F08FAFF300809E6AC42143
:100B0000818A46EE2C230020CC3D0008014B187052
:100B1000704700BF38230020F0B5334B1C7B85B0F5
:100B200034B1324B0E221A810024204605B0F0BDAC
:100B30002F4A1068516802AB03C308232D492E4881
:100B40000DEB030203F018F9054630B9274B2B488B
:100B50000A221A8100F0DAFCE6E70169B1F5702F8C
:100B600006D9224B26480B221A8100F0CFFCDCE785
:100B7000438B40F20A42934207D01C490C20088163
:100B80001946204800F0C2FCCFE71F4A024402F198
:100B90001003994204D2154B1C4810221A81E4E735
:100BA00010398E1A2046144900F0FAFC32460746E6
:100BB00005F11801204600F0F3FCAB689F4202D11A
:100BC000EB6898420AD0094B0D221A810090D5E9B2
:100BD00002123B460E4800F099FCA5E70D4800F0D4
:100BE00095FC0124A1E700BF683300202C230020DE
:100BF000793E0008DCFF0E0000000108E83D000817
:100C0000F43D0008063E00080800FFF7243E0008F7
:100C1000413E00086A3E00082DE9F04FADB006AF36
:100C200080460C4600F030FF054600285AD1237E4E
:100C3000022B1BD1E38A012B18D100F0ADFC064634
:100C4000FFF7AAFD03464FF4C870DFF8D092B3FB5C
:100C5000F0F206F5167602FB103316FA83F3C9F8A4
:100C60000030E37E33B9A84B00221A709C37BD4692
:100C7000BDE8F08FA38AEEB2013BB34205F1010556
:100C80000BD93B1D1E44E90000960023082201F009
:100C9000F801204601F00EF8ECE707F11400FFF729
:100CA00093FD324607F11401381D03F055F8002872
:100CB000D9D10F2E08D8944B1E70D9F80030A3F567
:100CC0001673C9F80030D1E7FB1CF8700146009399
:100CD00007220346204600F0EDFFF978404600F079
:100CE000CBFEC3E7E38A282B26D010D8012B1ED0D9
:100CF000052BBBD1BFF34F8F8449854BCA6802F4E3
:100D0000E0621343CB60BFF34F8F00BFFDE7302B92
:100D1000ACD1637E7F4D01336A7BDBB29342E946FF
:100D200003D1E27E2B7B9A4265D0CD469EE72146D9
:100D30004046FFF723FE99E7A38A013B9BB2C92BEC
:100D400094D8744D2E7B26BB05F10C03009308222A
:100D500033463146204600F0ADFF731CF2B2D90095
:100D60001E46A38A013B9A4205DA0E322A440092BB
:100D700000230822EEE700230022C5E90023002318
:100D8000AB6085F8D730C5F8D8302B7B0BB9E37E44
:100D90002B73002507F114093B1D082229464846FC
:100DA000C7E90155FD6001F0C1F83B7A05F1010A80
:100DB000AB424FEACA0608D9FB6808222B443146E9
:100DC000484601F0B3F85546EFE7C6F3CF06E17E9B
:100DD000CDE9049600230393A37E029319342823BC
:100DE0000093019446A3D3E90023404600F0B6FEE9
:100DF000FFF7FAFC3AE74FF0000807F11403A7F8F1
:100E000014801022009341460123204600F052FF37
:100E1000A68A023EB6B2F31C9B109B000733DB0888
:100E2000A9EBC3039D460DF1180A1FFA88F34FEA98
:100E3000C801B34201F110010AD20AEB0803009382
:100E400008220023204600F035FF08F10108ECE7F6
:100E500095F8D70000F0C8FAD5F8D83004461BB989
:100E600095F8D70000F0D0FAD5F8D83033449C423A
:100E700004D295F8D700013000F0C6FA4FEA960B7D
:100E80004FF000081FFA88F18B45D5E9003209D9E7
:100E90000AEB880103EB8800012200F0F3FA08F165
:100EA0000108EFE7F31842F10002C5E90032D5F876
:100EB000D83095F8D70006EB0308C5F8D88000F0C5
:100EC00093FA804509D395F8D730D5F8D800013387
:100ED000001B85F8D730C5F8D800FF2E08D80023AE
:100EE0002B7300F0A3FAFFF717FE08B1FFF70AFC17
:100EF0002B68094A9B0A013313810023AB6014E776
:100F000026417272DF25D7B73D33002000ED00E0A7
:100F10000400FA05683300202C2300204033002011
:100F200030B54FF00054244B22689A4285B007D068
:100F300002F0D8FB0446A8B90024204605B030BD15
:100F40001E4B627D1A701E48237D03731D49C92202
:100F50000E3000F07DFA2046E022002100F08AFAEF
:100F60000124EAE7184A194D136C43F00073136427
:100F7000AA6D174B9A42DFD12B6E013B7E2BDBD83B
:100F8000144A07CA01AB83E807001846032100F0A2
:100F90001DFB6B6D83424FF00003CDD12A6D8A4259
:100FA00001BFAB65054B2A6E1A7003BF0A4BEA6D91
:100FB0001A601C46C1E700BF9AAD44C53823002023
:100FC0006833002016000020003802400066004010
:100FD0005041A0B058660040182300202DE9FF477B
:100FE0004B4C02236371002302934A4BD3F800C099
:100FF000BCF57A7F12D3484B484FB7FBFCF69C45B3
:101000008CBF0A231123581EB6FBF3F503FB1562B0
:10101000C1B2002A3ED002280346F4D89DF80B3016
:101020003F4940485A1E9DF80A30013B1B0443EAE1
:101030000253BDF80820013A13434B6001F0F0FC65
:1010400000230193384B394900933948394B4FF409
:10105000805200F0EBFC384B197811B1344800F0A5
:101060000BFD00F099FA0546FFF796FB4FF4C873A5
:10107000B0FBF3F202FB130305F5167010FA83F0D0
:101080002E4B186002F024FB08B10F23238104B01B
:10109000BDE8F0876B1EB3F5806FBFD2C1EBC10E08
:1010A0000EF103034FEAE309C3F3C703A1EB0308FF
:1010B00009F1010A4FF47A705FFA88F609FB000023
:1010C0005AFA88F8B0FBF8F0B0F5617F08D90EF154
:1010D000FF33C3F3C703C91ACEB2591E0F2914D860
:1010E000721E072A8CBF00220122991901FB0551AB
:1010F000B7FBF1F7BC4591D1002A8FD0ADF808506D
:101100008DF80A308DF80B6088E71346EDE700BFD5
:101110002C230020182300203F420F0040787D013F
:101120001023002080340020850800083C23002084
:1011300044330020190C00083823002040330020DD
:101140002DE9F04F8EA7D7E900670FF23C29D9E9C6
:101150000089854D93B0DFF838B2844C284600F002
:1011600061FD0DF1300A079070B310220021504646
:1011700000F080F9079B197B4FF0000261F3030236
:101180008DF83020586899680EAA03C21B680D9A22
:1011900063F31C029DF830300D9243F020038DF86C
:1011A0003030002352461946584601F049FC07905A
:1011B00028B9284600F03AFD079B2370CEE7237834
:1011C000072B36D80133237018220021504600F037
:1011D00051F9DFF8BCB1002319465246584601F0D8
:1011E00057FC014648BB102208A800F043F900F064
:1011F000D5F90B4612A9024611E9030009AC84E8AF
:1012000003009DF83410C1F3030089064CBF0E9C07
:10121000BDF838408DF82C0046BFC4F31C0444F0E0
:101220000044C4F30A0408A92846089400F0C6FE46
:10123000D1E7284600F0FAFCC6E7284600F024FC77
:101240000446002848D1DFF84CB100F0A5F9DBF8DE
:101250000030984240D300F09FF90790FFF79CFAC6
:10126000079A8DF8204003464FF4C87002F51672B5
:10127000B3FBF0F101FB103312FA83F3CBF800302B
:10128000DFF814B19BF8001011B901238DF820305C
:1012900050460791FFF798FA0799C1F11004E4B29C
:1012A000062C28BF0624224651440DF1210000F0EF
:1012B000CFF808AB03931823029301342C4B01930E
:1012C000E4B20123009304943B463246284600F0E2
:1012D000DDFB00238BF8003000F05EF9254A264C38
:1012E0001368C31AB3F57A7F31D3106000F056F952
:1012F00002460B46284600F0A3FC284600F0C4FB3B
:1013000028B3237BDFF894B0002B14BF0323022300
:101310008BF8053000F040F94FF47A735146B0FB7A
:10132000F3F0CBF800005846FFF7F0FA1823073027
:101330000293124B0193C0F3CF0040F25513CDE955
:1013400003A0009342464B46284600F09FFB237BB8
:101350002BB1FFF749FA237B002B7FF4FCAE13B0CF
:10136000BDE8F08FAFF30080443300204D340020FF
:101370003C33002048340020683300204C340020E7
:10138000401DA12026812A0BF1C6A7C1D068080FF5
:1013900080340020403300203D3300202C230020E7
:1013A00070B501F0FDFF094E094D3080002428681A
:1013B0003388834208D901F0EDFF2B6804440133E0
:1013C000B4F5803F2B60F2D370BD00BF7C340020A9
:1013D0005034002002F092B800F10060920000F555
:1013E000803002F023B80000054B1A68054B1B88BB
:1013F0009B1A834202D9104401F0CCBF00207047F1
:10140000503400207C34002038B5074D044628684D
:10141000204401F0C7FF28B928682044BDE83840BF
:1014200001F0D8BF38BD00BF50340020064991F804
:10143000243033B10023086A81F824300822FFF7F2
:10144000CBBF0120704700BF54340020704700001C
:1014500010B50023934203D0CC5CC4540133F9E7A8
:1014600010BD000003460246D01A12F9011B0029E4
:10147000FAD1704702440346934202D003F8011B9D
:10148000FAE770472DE9F8431F4D144695F82420DC
:101490000746884652BBDFF870909CB395F824301D
:1014A0002BB92022FF2148462F62FFF7E3FF95F872
:1014B0002400C0F10802A24228BF2246D6B241460B
:1014C000920005EB8000FFF7C3FF95F82430A41BC2
:1014D0001E44F6B2082E17449044E4B285F8246006
:1014E000DBD1FFF7A3FF0028D7D108E02B6A03EB7D
:1014F00082038342CFD0FFF799FF0028CBD1002091
:10150000BDE8F8830120FBE7543400200FB400202D
:1015100004B0704700B59BB0EFF3098168226846BC
:10152000FFF796FFEFF30583044B9A6BDA6A9A6A2A
:101530009A6A9A6A9A6A9A6A9B6AFEE700ED00E0E4
:1015400000B59BB0EFF3098168226846FFF780FF82
:10155000EFF30583044B9A6B9A6A9A6A9A6A9A6ABD
:101560009A6A9B6AFEE700BF00ED00E000B59BB001
:10157000EFF3098168226846FFF76AFFEFF30583FE
:10158000034B5A6B9A6A9A6A9A6A9A6A9B6AFEE74E
:1015900000ED00E0FEE7000001F0EABF01F0C2BF8D
:1015A00030B5094D0A4491420DD011F8013B584025
:1015B000082340F30004013B2C4013F0FF0384EAAE
:1015C0005000F6D1EFE730BD2083B8EDF7B54FF00E
:1015D000FF33DFF854C0DFF854E000EB81011A4616
:1015E00088421CD050F8044B019401AF042417F832
:1015F000015B82EA05620825DB18164605F1FF3516
:101600005241002EBCBF83EA0C0382EA0E0215F0A1
:10161000FF05F1D1013C14F0FF04E8D1E0E7D84325
:10162000D14303B0F0BD00BF9336EAA9EBE1F0422D
:101630002DE9F041C56915B9C161BDE8F0814B687C
:1016400023F06047C3F38A464FEAD37EC3F3807822
:1016500016EA230638BF3E46AC462B465A68BEEB18
:10166000D27F22F060440AD0002A18DAA40CB442D7
:1016700017D19D420FD10D60DEE71346EEE7A7427A
:1016800007D102F08044C2F3807242450BD054B1BE
:10169000EFE708D2EDE7CCF800100B60CDE7B442DD
:1016A00001D0B442E5D81A689C46002AE5D11960F9
:1016B000C3E700002DE9F047089D01F007044FEA59
:1016C000D508224405F0070500EBD1004FF47F490F
:1016D000944201D1BDE8F08704F0070705F0070A3E
:1016E00057453E4638BF5646C6F10806111B8E4286
:1016F00028BF0E46E10808EBD50E415C13F80EC07A
:10170000B94029FA06F721FA0AF1FFB28CEA010181
:1017100047FA0AF739408CEA010C03F80EC034444A
:101720003544D5E780EA0120082341F2210201B2C5
:101730004000002980B203F1FF33B8BF504013F0DE
:10174000FF03F4D17047000038B50C468D18A54250
:1017500000D138BD14F8011BFFF7E4FFF7E70000E4
:1017600002684AB113680360C388018901339BB2E0
:101770009942C38038BF03811046704770B588B066
:10178000202204460D4668460021FFF773FE2046DE
:101790000495FFF7E5FF024658B16B46054608AED3
:1017A0001C4603CCB44228606960234605F1080555
:1017B000F6D1104608B070BD10B54B6823B9CA8A7F
:1017C00063F30902CA8210BDC4681A681C60C36052
:1017D000438A013B43824A60EFE700002DE9F84F5E
:1017E0001D46CB8A0F46C3F309010629814692465E
:1017F0000B4630D00020AAB207F119049EB2052E84
:101800001FFA80F80FD8904503F1010306D3FB8A35
:101810000A4462F30903FB8201201AE01AF800600F
:10182000E6540130EAE79045F1D2A1F1060B1C2302
:101830007C68BBFBF3F203FB12BB1FFA8BF6002C98
:1018400045D14846FFF78CFF044638B978606FF001
:101850000200BDE8F88F4FF00008E6E700260660BA
:101860007860ADB24FF0000B454510D90AEB080384
:10187000221D13F8011B9155B1B208F101081B2973
:101880001FFA88F82BD0454506F10106F1D8FB8AEE
:10189000C3F30902154465F30903BCE7013292B2B0
:1018A0001C462368002BF9D1AB1F0B441C21B3FB52
:1018B000F1F301339BB29A42D3D2BBF1000FD0D1E6
:1018C0004846FFF74DFF20B9C4F800B0BFE701223A
:1018D000E7E7C0F800B05E4620600446C1E7454532
:1018E000D5D94846FFF73CFF08B92060AFE7C0F8FC
:1018F00000B0002620600446B6E700002DE9F04F56
:101900002DED028B83B0CDE90013BDF83C4080463D
:101910009246002A00F087802CB10E9B002B00F02D
:101920008280072C2BD808F10C00FFF719FF054621
:1019300038B96FF00205284603B0BDEC028BBDE854
:10194000F08F14220021FFF795FD22460E9905F134
:101950000800FFF77DFD631C2B749AF800302C44BF
:1019600003F01F0363F03F032372009B43F0004129
:10197000696040462946FFF75BFE0125DBE700F181
:101980000C034FF0000908EE103A4FF0800B4E4662
:101990004D4618EE100AFFF7E3FE07460028C8D0B0
:1019A00014220021FFF766FD002E3AD1019B3B81F6
:1019B00002220E9B02F1080103EB060C57FA81F19B
:1019C0001046B44202F10102D2B201D8024607E049
:1019D0001CF8010B01F8010B0136062AB6B2EFD94B
:1019E0009AF8001001F01F01B44208BF4FF0400BFD
:1019F000B81841EA49114BEA01030372009B013216
:101A000043F000437B603A7439464046FFF710FECE
:101A10000135B4422DB289F001094FF0000BB8D165
:101A200089E70022C5E76FF0010584E7F8B51546A0
:101A30000E462422002104461F46FFF71BFD069B8D
:101A40006360B5F5001F079BA76034BF6A094FF6B6
:101A5000FF72236204F10C0097B200239A4205D86A
:101A60000023036027826382A382F8BD06600133EE
:101A700030462036F2E7000003781BB94BB2002B4A
:101A8000C8BF017070470000007870472DE9F74F1C
:101A9000DDF83C90BDF830500D9E9DF83840BDF803
:101AA0004070804692469B46B9F1000F01D1002F4D
:101AB00051D11F2C4FD898F80000B0B9072F47D844
:101AC00035F0030347D13A4649464FF6FF70FFF71A
:101AD0003BFE20F001002D02400445EA0464400C66
:101AE00044EA40244FF6FF7321E040EA0520072F27
:101AF00040EA0464F6D900254FF6FF73C5F12000D3
:101B0000A5F120022AFA05F10BFA00F001432BFAA5
:101B100002F211431846C9B2FFF704FE0835402D02
:101B20000346EBD13A464946FFF70EFE0346CDE9A0
:101B30000097324621464046FFF7E0FE33780133F6
:101B4000DBB21F2B88BF0023337003B0BDE8F08FDA
:101B50006FF00300F9E76FF00100F6E72DE9F04FB1
:101B600085B09246DDF848800F9D9DF840209DF895
:101B70004490BDF84C7006469B46B8F1000F01D169
:101B8000002F48D11F2A46D83378002B46D00C02AC
:101B900044EA02649DF8381044EAC93444EA014436
:101BA0001C43072F44F0800432D900234FF6FF7204
:101BB000C3F1200CA3F120002AFA03F10BFA0CFC6C
:101BC00041EA0C012BFA00F00143C9B2104603931D
:101BD000FFF7A8FD039B0833402B0246E8D13A46A5
:101BE0004146FFF7B1FD0346CDE900872A4621466D
:101BF0003046FFF783FEB9F1010F06D12B78013390
:101C0000DBB21F2B88BF00232B7005B0BDE8F08F1F
:101C10004FF6FF73E8E76FF00100F6E76FF003009F
:101C2000F3E70000C06900B104307047C3691A6867
:101C3000C261C2681A60C360438A013B4382704735
:101C40002DE9F041D0F81880194E14461D46414642
:101C5000002709B9BDE8F081D1E90223A21A65EB9A
:101C60000303964277EB03031ED283698B420DD1A7
:101C7000FFF7A2FD83691B688361C3680B60438A19
:101C8000C1608169013B43828846E2E7FFF794FD2A
:101C90000B68C8F80030C3680B60438AC160013B21
:101CA0004382D8F80010D4E788460968D1E700BF1E
:101CB00080841E002DE9F04F8BB00D46DDF850906A
:101CC00014469B468046002800F01981B9F1000FA8
:101CD00000F01581531E3F2B00F21181012A03D120
:101CE000BBF1000F40F00B810023CDE90833B8F8B9
:101CF0001430B5EBC30F4FEAC30703D300200BB07A
:101D0000BDE8F08F2B199F42D8F80C303ABF7F1BEB
:101D1000FFB227461BB9D8F81030002B7AD02F2DF0
:101D20004ED8C5F13006B7424FF000032CBFF6B2D3
:101D30003E4600932946D8F8080008AB3246FFF724
:101D4000B9FCA7EB060A35445FFA8AFAB8F81430F2
:101D500003F10053063BDB000493D8F80C300393E7
:101D60003021039B13B1BAF1000F2CD1D8F8100029
:101D700040B1BAF1000F05D0009608AB5246691A7F
:101D8000FFF798FC38B2002FB8D066070AD00AAB2C
:101D900003EBD401624211F8083C02F00702134140
:101DA00001F8083C082C3CD9102C40F2B580202CBE
:101DB00040F2B780BBF1000F00F09C80082334E0B4
:101DC000BA460026C2E7049BE02B28BFE023069317
:101DD0000B44AB42059314D95A1B039800969245C5
:101DE00034BF5246D2B2691A08AB04300792FFF7EB
:101DF00061FC079A1644AAEB020A1544F6B25FFA90
:101E00008AFA049B069A05999B1A0493039B1B6804
:101E10000393A6E70093D8F8080008AB3A46294692
:101E2000AEE7BBF1000F13D00123B4EBC30F6CD0AE
:101E3000082C12D89DF82030621E23FA02F2D50732
:101E400006D54FF0FF3202FA04F423438DF8203018
:101E50009DF8203089F8003051E7102C12D8BDF8D9
:101E60002030621E23FA02F2D10706D54FF0FF326E
:101E700002FA04F42343ADF82030BDF82030A9F86D
:101E800000303CE7202C0FD80899631E21FA03F399
:101E9000DA0705D54FF0FF3202FA04F40C43089438
:101EA000089BC9F800302AE7402C2BD0DDE90865F3
:101EB000611EC4F12102A4F1210326FA01F105FA01
:101EC00002F225FA03F311431943CB0712D501227D
:101ED000A4F12003C4F1200102FA03F322FA01F174
:101EE000A240524243EA010363EB430332432B43D4
:101EF000CDE90823DDE90823C9E90023FFE66FF0F7
:101F00000100FCE66FF00800F9E6082CA0D9102CBF
:101F1000B3D9202CEED8C3E7BBF1000FADD002231C
:101F200083E7BBF1000FBBD004237EE730B5012A65
:101F3000144638BF0124402C85B028BF402400251A
:101F4000012ACDE9025518D81B788DF808306307AF
:101F50000AD004AB03EBD405624215F8083C02F04A
:101F60000702934005F8083C0091034622460021F1
:101F700002A8FFF79FFB05B030BD082AE4D9102A5C
:101F800003D81B88ADF80830E1E7202A8DBFD3E9DC
:101F900000231B680293CDE90223D8E710B5CB6874
:101FA0001BB98B600B618B8210BDC4681A681C6002
:101FB000C360438A013B4382CA60F0E72DE9F04FDA
:101FC000D1F8008093B018F0800FCDE90323C8F357
:101FD000C01219BFC8F3C03BC8F306264FF0020B6E
:101FE0001646B8F1000F04460D4680F2C58118F080
:101FF000C043059340F0C0810B7B002B00F0BC81F7
:10200000BBF1020F03D00178B14240F0B88108F073
:102010007F0106916AB3C8F3074A2B44069A93F8E6
:102020000390760646EA0B4646EA82465FEAD913F3
:1020300046EA0A06079300F0908000220023CDE9CB
:102040000A23069B009367685B4652460AA920460E
:10205000B84700287ED0A7699FB9314604F10C002B
:10206000FFF78CFB0746E0B96FF0020013B0BDE844
:10207000F08FC8F30F2A18F07F0F08BF0AF0030A89
:10208000CBE73B699E420DD03F68002FF9D1314626
:1020900004F10C00FFF772FB07460028E4D0A369A7
:1020A0003B60A761DDE90A2300264FF6FF70C6F109
:1020B000200E22FA06F103FA0EFEA6F1200C23FAF6
:1020C0000CFC41EA0E0141EA0C01C9B20836099242
:1020D0000893FFF727FB402EDDE90832E7D1B882ED
:1020E000FB7D09F01F06C3F384039B1BD7E9022184
:1020F00098B2002BBCBF00F120031BB252EA0100D2
:10210000C8F304680FD00398821A049860EB0101A9
:10211000A14890424FF000028A4104D3079A002A56
:1021200055D0012B23DDFA7D4FEA890302F003022B
:1021300003F07C031343FB7539462046FFF73CFB55
:10214000079BA3B9FB7DC3F38402013262F38603CC
:10215000FB7504E06FF00B0088E7A76917B96FF013
:102160000C0083E73B699E42BAD03F68F6E719F05E
:10217000400F2CD0039BBB60049BFB60142200210A
:102180000DA8FFF777F9039B0A93049B0B932B1D74
:102190000C932B7BADF83EA0013BDBB2ADF83C309D
:1021A000069B8DF843308DF840B0A3688DF84160F0
:1021B0008DF842800AA920469847FB7DC3F384032B
:1021C000013303F01F039B02FB8200204EE7FB7DDF
:1021D000C9F34012B2EBD31F40F0D480C3F38403A1
:1021E000B34240F0D28007992B7B4FEA9912002925
:1021F00034D0D20741D4032B40F2CA80039BBB608A
:10220000049BFB602B7BAE1D033BDBB232463946A1
:1022100004F10C00FFF7E2FA00280DDA20463946F7
:10222000FFF7CAFAFB7DC3F38403013303F01F03F6
:102230009B02FB82032019E7AB883B832A7B033A8E
:10224000B88AD2B23146FFF77FFAFB7DB882DA4313
:10225000C2F3C01262F3C713FB75B6E76AB92E1D4D
:10226000013BDBB23246394604F10C00FFF7B6FA07
:102270000028D3DB2A7B013AE2E7F98AC1F309019E
:10228000013B0529DAB253D8281D002307F11A0CA7
:102290009A4208D910F801EB0CF801E00131013342
:1022A0000629DBB2F4D103990A9104990B91934268
:1022B00007F11A010C9138BF043379680D9134BFCE
:1022C00055FA83F300230E93FB8AADF83EA0C3F3C7
:1022D00009031A44069B8DF843300023ADF83C20D7
:1022E0008DF840B08DF841608DF842807B602A7B8C
:1022F000B88A013A291DFFF727FA3B8BB88283423F
:1023000003D1A3680AA92046984720460AA9FFF7E7
:1023100045FEFB7DB88AC3F38403013303F01F033A
:102320009B02FB823B8B984214BF112000209DE64C
:102330007B68002BB7D0062001E01C306346D3F841
:1023400000C0BCF1000FF8D1091A081D05F1040CFA
:1023500000EB030905989DF8143001EB000EBEF167
:102360001B0FA0D89A429ED91CF8013B09F8013BEB
:10237000059B01330593EDE76FF0090076E66FF0FA
:102380000A0073E66FF00D0070E66FF00E006DE668
:102390006FF00F006AE600BF80841E00404BF0B56E
:1023A0001C6C404E44F000741C641D6E45F00075BA
:1023B0001D661B6E3C4B9B6AD3F80052354045F0BE
:1023C0000105C3F80052D3F80042344044EA00202B
:1023D00040F00100C3F80002002952D00020C3F8E9
:1023E0001C020546C3F80402C3F80C02C3F8140229
:1023F00003EBC00401301C28C4F84052C4F8445216
:10240000F6D100254FF0010C96781488F70748BFE5
:10241000D3F804720CFA04F044BF0743C3F8047203
:10242000B70742BFD3F80C720743C3F80C727607A4
:1024300042BFD3F814620643C3F8146203EBC4042A
:102440005668C4F840629668C4F84462D3F81C42E7
:1024500001352043A942C3F81C0202F10C02D3D17A
:10246000D3F8002222F00102C3F800220C4B1A6CB0
:1024700022F000721A641A6E22F000721A661B6E45
:10248000F0BD0122C3F84012C3F84412C3F804128D
:10249000C3F81412C3F80C22C3F81C22E0E700BFF3
:1024A000003802400000FFFF80340020184A916A83
:1024B00008B58B688B6013F0010104D013F00C0F8A
:1024C00018BF4FF48031D80506D513F4406F14BF00
:1024D00041F4003141F00201D80306D513F4402F36
:1024E00014BF41F4802141F00401D3690BB10848C5
:1024F0009847202383F311880648002100F016FE38
:10250000002383F31188BDE8084001F029B900BF1A
:10251000803400208834002038B5124CA36ADD686E
:10252000AA0712D05A6922F002025A61A36913B1B4
:10253000012120469847202383F311880A4800216F
:1025400000F0F4FD002383F31188EB0606D5A36A9F
:102550001021D960236A0BB102489847BDE8384082
:1025600001F0FEB8803400209034002038B5124CC1
:10257000A36A1D69AA0712D05A6922F010025A6193
:10258000A36913B1022120469847202383F31188C1
:102590000A48002100F0CAFD002383F31188EB06EE
:1025A00006D5A36A10211961236A0BB10248984726
:1025B000BDE8384001F0D4B88034002090340020C9
:1025C00038B50F4CA36A5D685D602A070AD50422FE
:1025D00022701A6822F002021A60636A13B10021A5
:1025E000204698476B0706D5A36A9969236A13B1F9
:1025F000034809049847BDE8384001F0B1B800BF6E
:102600008034002010B50E4C204600F0F7F90D4B39
:10261000A3620B21132000F0D9F90B21142000F044
:10262000D5F90B21152000F0D1F90B21162000F06F
:10263000CDF90022BDE8104011460E20FFF7AEBED6
:102640008034002000640040114B984210B50446CD
:1026500009D1104B1A6C42F000721A641A6E42F0E3
:1026600000721A661B6EA36A01221A60A36A5A6876
:10267000D20707D5626851681268D9611A60064AA4
:102680005A6110BD0121082000F046FCEEE700BFB2
:1026900080340020003802405B87010003291AD8EB
:1026A000DFE801F0020A0F14836A9B6813F0E05F11
:1026B00014BF012000207047836A9868C0F38060CF
:1026C0007047836A9868C0F3C0607047836A9868EF
:1026D000C0F30070704700207047000010B5032958
:1026E00025D8DFE801F00225292D836A9968C1F316
:1026F0000161183103EB0113107884064CBF546854
:102700009488C0F300114FEA410148BF41EAC40177
:1027100000F00F004CBF41F0040141EA4451586001
:1027200041F001019068D2689860DA60196010BDCC
:10273000836A03F5C073DFE7836A03F5C873DBE7D9
:10274000836A03F5D073D7E701290AD002290FD095
:1027500081B9836ADA68920701D1186903E0012020
:102760007047836AD86810F0030018BF01207047D3
:10277000836AF2E70020704710B539B9836AD968D7
:1027800089071BD11B699C0704D110BD012915D0F5
:102790000229FAD1816AD1F8C031D1F8C441D1F807
:1027A000C8011061D1F8CC0150612020086108698E
:1027B000800717D1486940F0100012E0816AD1F813
:1027C000B031D1F8B441D1F8B8011061D1F8BC01F1
:1027D00050612020C860C868800703D1486940F074
:1027E00002004861C3F34000C3F38001000140EAE6
:1027F0004111107920F030000143117189064BBF5F
:1028000091681189DB085B0D4CBF63F31C0163F316
:102810000A01137948BF916064F3030313714FEA0F
:1028200014234FEA144458BF118113705480ACE74D
:10283000026843681143016003B118477047000004
:10284000024AD36843F0C003D360704700100140D0
:10285000024AD36843F0C003D3607047004400408D
:102860002DE9F041D0F85C62F7683368DA05044678
:102870009DB20DD5202383F311884FF400710430ED
:10288000FFF7D6FF6FF480733360002383F3118862
:10289000202383F3118804F1040815F02F033AD1A3
:1028A00083F31188380615D5290613D5202383F321
:1028B000118804F1380000F023FA00284DDA0821CD
:1028C000201DFFF7B5FF4FF67F733B40F3600023F9
:1028D00083F311887A0616D56B0614D5202383F36B
:1028E0001188D4E913239A420AD1236C43B127F00B
:1028F00040073F041021201D3F0CFFF799FFF760B0
:10290000002383F31188D4F86422D3683BB3BDE875
:10291000F041106918472B0713D015F0080F0CBFB2
:1029200000218021E80748BF41F02001AA0748BFE5
:1029300041F040016B0748BF41F480714046FFF70A
:1029400077FFAD06736805D594F8601220461940EC
:1029500000F078FA3568ADB29FE77060B7E7BDE880
:10296000F081000008B50348FFF77AFFBDE8084092
:1029700000F0F6BEAC34002008B50348FFF770FF46
:10298000BDE8084000F0ECBE1437002010B5094C3B
:10299000094A2046002100F033FA084BC4F85C32A3
:1029A000074C084A0021204600F02AFA064BC4F8DA
:1029B0005C3210BDAC3400204128000800100140FA
:1029C00014370020512800080044004000F1604303
:1029D00003F561430901C9B283F80013012200F035
:1029E0001F039A4043099B0003F1604303F56143D1
:1029F000C3F880211A607047FFF704BE012300F17D
:102A00000802C0E90222037000F110020023C0E9AD
:102A10000422C0E90633C0E9083343607047000070
:102A200010B52023044683F311880223037041600C
:102A3000FFF70AFE04232370002383F3118810BDDF
:102A40002DE9F0411F4604460D461646202383F328
:102A5000118800F108082378052B0DD0294620465F
:102A6000FFF71CFE40B1204632462946FFF736FEEE
:102A7000002080F3118808E03946404600F03AFB18
:102A80000028E8D0002383F31188BDE8F08100001E
:102A90002DE9F0411F4604460D461646202383F3D8
:102AA000118800F110082378052B0DD02946204607
:102AB000FFF74AFE40B1204632462946FFF75CFE4A
:102AC000002080F3118808E03946404600F012FBF0
:102AD0000028E8D0002383F31188BDE8F0810000CE
:102AE000F8B5154682680669AA420B46816938BF67
:102AF0008568761AB54204460BD218462A46FEF778
:102B0000A7FCA3692B44A361A3685B1BA3602846B1
:102B1000F8BD0CD918463246FEF79AFCAF1BE168A7
:102B20003A463044FEF794FCE3683B44EBE7184632
:102B30002A46FEF78DFCE368E5E7000083689342D0
:102B4000F7B51546044638BF8568D0E90460361AE3
:102B5000B5420BD22A46FEF77BFC63692B446361C6
:102B6000A36828465B1BA36003B0F0BD0DD93246B5
:102B70000191FEF76DFC0199E068AF1B3A463144C4
:102B8000FEF766FCE3683B44E9E72A46FEF760FC93
:102B9000E368E4E710B50A440024C361029B846043
:102BA000C0E90000C0E90511C1600261036210BD07
:102BB00008B5D0E90532934201D1826882B98268B2
:102BC000013282605A1C42611970D0E904329A4283
:102BD00024BFC3684361002100F09CFA002008BDB7
:102BE0004FF0FF30FBE7000070B5202304460E468F
:102BF00083F31188A568A5B1A368A269013BA3600E
:102C0000531CA36115782269934224BFE368A36132
:102C1000E3690BB120469847002383F311882846C7
:102C200007E03146204600F065FA0028E2DA85F335
:102C3000118870BD2DE9F74F04460E461746984699
:102C4000D0F81C904FF0200A8AF311884FF0000B47
:102C5000154665B12A4631462046FFF741FF034637
:102C600060B94146204600F045FA0028F1D0002323
:102C700083F31188781B03B0BDE8F08FB9F1000F22
:102C800003D001902046C847019B8BF31188ED1AB1
:102C90001E448AF31188DCE7C0E90511C160C361F5
:102CA0001144009B8260C0E900000161036270472B
:102CB000F8B504460D461646202383F31188A7680D
:102CC000A7B1A368013BA36063695A1C62611D70D0
:102CD000D4E904329A4224BFE3686361E3690BB12B
:102CE00020469847002080F3118807E031462046AF
:102CF00000F000FA0028E2DA87F31188F8BD00003E
:102D0000D0E905239A4210B501D182687AB9826868
:102D1000013282605A1C82611C7803699A4224BF86
:102D2000C3688361002100F0F5F9204610BD4FF023
:102D3000FF30FBE72DE9F74F04460E46174698464D
:102D4000D0F81C904FF0200A8AF311884FF0000B46
:102D5000154665B12A4631462046FFF7EFFE034689
:102D600060B94146204600F0C5F90028F1D00023A3
:102D700083F31188781B03B0BDE8F08FB9F1000F21
:102D800003D001902046C847019B8BF31188ED1AB0
:102D90001E448AF31188DCE702684368114301602E
:102DA00003B11847704700001430FFF743BF00001D
:102DB0004FF0FF331430FFF73DBF00003830FFF70E
:102DC000B9BF00004FF0FF333830FFF7B3BF00004A
:102DD0001430FFF709BF00004FF0FF311430FFF748
:102DE00003BF00003830FFF763BF00004FF0FF3231
:102DF0003830FFF75DBF000000207047FFF7C6BD09
:102E000037B515460E4A026000224260C0E9022230
:102E10000122044602740B46009000F15C014FF45D
:102E200080721430FFF7B6FE00942B464FF4807288
:102E300004F5AE7104F13800FFF72EFF03B030BD8A
:102E4000843E000838B5C36904460D461BB9042109
:102E50000844FFF7A1FF294604F11400FFF7A8FE7C
:102E6000002806DA201D4FF48061BDE83840FFF7E6
:102E700093BF38BD024B0022C3E900339A6070470C
:102E80007C390020002303748268054B1B68996815
:102E90009142FBD25A6803604260106058607047EC
:102EA0007C39002008B5202383F31188037C032B91
:102EB00005D0042B0DD02BB983F3118808BD4369CD
:102EC00000221A604FF0FF334361FFF7DBFF00235E
:102ED000F2E7D0E9003213605A60F3E7002303748D
:102EE0008268054B1B6899689142FBD85A68036059
:102EF00042601060586070477C390020054B1969AA
:102F00000874186802681A6053601861012303741A
:102F1000FDF77EBB7C39002030B54B1C0B4D87B0D4
:102F2000044610D02B690A4A01A800F01BF920467C
:102F3000FFF7E4FF049B13B101A800F04FF92B69E0
:102F4000586907B030BDFFF7D9FFF8E77C3900209A
:102F5000A52E000838B50C4D41612B6981689A682F
:102F60009142044603D8BDE83840FFF78BBF1846AE
:102F7000FFF7B4FF01232C61014623742046BDE80E
:102F80003840FDF745BB00BF7C390020044B1A6870
:102F90001B6990689B68984294BF0020012070478D
:102FA0007C39002010B5084C236820691A6822601B
:102FB0005460012223611A74FFF790FF01462069D3
:102FC000BDE81040FDF724BB7C39002008B5FFF7B1
:102FD000DDFF18B1BDE80840FFF7E4BF08BD000001
:102FE000FFF7E0BFFEE7000010B50C4CFFF742FF13
:102FF00000F0AAF80A498022204600F031F80123A7
:1030000044F8180C037400F087FB002383F3118845
:1030100062B60448BDE8104000F042B8A439002070
:10302000AC3E0008BC3E000800F012B9EFF311807E
:1030300020B9EFF30583202282F311887047000046
:1030400010B530B9EFF30584C4F3080414B180F36C
:10305000118810BDFFF7BAFF84F31188F9E700006B
:1030600082600222028270478368A3F17C0243F8E7
:103070000C2C026943F83C2C426943F8382C074A6F
:1030800043F81C2CC26843F8102C022203F8082CC9
:10309000002203F8072CA3F1180070472906000846
:1030A00010B5202383F31188FFF7DEFF00210446CB
:1030B000FFF750FF002383F31188204610BD000066
:1030C000024B1B6958610F20FFF718BF7C390020A5
:1030D000202383F31188FFF7F3BF000008B50146F2
:1030E000202383F311880820FFF716FF002383F3C2
:1030F000118808BD49B1064B42681B6918605A60C7
:10310000136043600420FFF707BF4FF0FF307047A4
:103110007C3900200368984206D01A68026050602B
:1031200059611846FFF7AEBE7047000038B5044637
:103130000D462068844200D138BD036823605C607E
:103140004561FFF79FFEF4E7054B03F11402C3E965
:1031500005224FF0FF310022C3E90712704700BF7C
:103160007C39002070B51C4EC0E9032305460C468F
:1031700000F058FB334653F8142F9A420DD13062B9
:10318000C5E901242A600A2C2CBF00190A30C6E9BF
:103190000555BDE8704000F033BB316A431AE318AF
:1031A00038BF1C469368A34202D9081900F036FBC9
:1031B00073699A6894420CD85A68AC602B606A6054
:1031C00015609A685D60121B9A604FF0FF33F361DF
:1031D00070BD1B68A41AECE77C39002038B51B4C85
:1031E000636998420DD0D0E9003213605A60002222
:1031F0008168C2609A680A449A604FF0FF33E361C5
:1032000038BD2246036842F8143F002193425A60B9
:10321000C16003D1BDE8384000F0FABA9A6881680D
:10322000256A0A449A6000F0FDFA63699A68411BB6
:103230008A42E5D9AB181D1A092D206A98BF01F101
:103240000A02BDE83840104400F0E8BA7C3900209A
:103250002DE9F041184C002704F11406656900F0CF
:10326000E1FA236AAA68C11A8A4215D81344236274
:10327000D5E9003213605A606369D5F80C80EF60BD
:10328000B34201D100F0C4FA87F311882869C0471E
:10329000202383F31188E1E76169B14209D0134427
:1032A0001B1ABDE8F0410A2B2CBFC0180A3000F0F1
:1032B000B5BABDE8F08100BF7C390020002070471E
:1032C000FEE70000704700004FF0FF30704700003D
:1032D000BFF34F8F024AD368DB03FCD4704700BFB3
:1032E000003C024008B5094B1B7873B9FFF7F0FFAB
:1032F000074B1A69002ABFBF064A5A6002F188329A
:103300005A601A6822F480621A6008BD383B0020B7
:10331000003C02402301674508B50B4B1B7893B96D
:10332000FFF7D6FF094B1A6942F000421A611A688A
:1033300042F480521A601A6822F480521A601A68A5
:1033400042F480621A6008BD383B0020003C024015
:103350000B28F0B516D80C4C0C4923787BB90C4DD2
:103360000E460C234FF0006255F8047B46F8042B00
:10337000013B13F0FF033A44F6D10123237051F8C7
:103380002000F0BD0020FCE76C3B00203C3B00200F
:10339000D43E0008014B53F820007047D43E00088B
:1033A0000C2070470B2810B5044601D9002010BD31
:1033B000FFF7CEFF064B53F824301844C21A0BB95E
:1033C0000120F4E712680132F0D1043BF6E700BFB8
:1033D000D43E00080B2810B5044621D8FFF778FF2B
:1033E000FFF780FF0F4AF323D360C300DBB243F43F
:1033F000007343F002031361136943F480331361D4
:10340000FFF766FFFFF7A4FF074B53F8241000F007
:1034100029F9FFF781FF2046BDE81040FFF7C2BF42
:10342000002010BD003C0240D43E0008F8B512F068
:103430000103144642D18218B2F1016F57D82D4BC7
:103440001B6813F0010352D02B4DFFF74BFFF32302
:10345000EB60FFF73DFF40F20127032C15D824F065
:1034600001046618244C401A40F20117B142236946
:1034700000EB010524D123F001032361FFF74CFF8A
:103480000120F8BD043C0430E7E78307E7D12B694E
:1034900023F440732B612B693B432B6151F8046B80
:1034A0000660BFF34F8FFFF713FF03689E42E9D01A
:1034B0002B6923F001032B61FFF72EFF0020E0E7CB
:1034C00023F44073236123693B4323610B882B80E2
:1034D000BFF34F8FFFF7FCFE2D8831F8023BADB2F2
:1034E000AB42C3D0236923F001032361E4E718460C
:1034F000C7E700BF00380240003C0240084908B559
:103500000B7828B11BB9FFF7EDFE01230B7008BD46
:10351000002BFCD0BDE808400870FFF7FDBE00BFDF
:10352000383B002070B582B0FFF780FD0E4E054697
:1035300000F078F93268904237BF0C4A0B49516865
:1035400014682EBFD1E900410131516004190346CE
:1035500041F10001284601913360FFF771FD0199A7
:10356000204602B070BD00BF703B0020783B0020B9
:1035700070B582B0FFF75AFD104E054600F052F9C3
:103580003268904237BF0E4A0D49516814682EBF09
:10359000D1E9004101315160041941F100010346B4
:1035A000284601913360FFF74BFD01994FF47A7281
:1035B00000232046FCF714FE02B070BD703B0020D3
:1035C000783B002010B50244064BD2B2904200D1A5
:1035D00010BD441C00B253F8200041F8040BE0B2C7
:1035E000F4E700BF502800400F4B30B51C6F240497
:1035F00007D41C6F44F400741C671C6F44F400442F
:103600001C670A4C236843F4807323600244084B10
:10361000D2B2904200D130BD441C00B251F8045BDC
:1036200043F82050E0B2F4E7003802400070004058
:103630005028004007B5012201A90020FFF7C2FF72
:10364000019803B05DF804FB13B50446FFF7F2FFE1
:10365000A04205D0012201A900200194FFF7C4FF78
:1036600002B010BD70470000074B45F255521A607A
:1036700002225A6040F6FF729A604CF6CC421A6001
:10368000024B01221A70704700300040843B00203A
:10369000034B1B781BB1034B4AF6AA221A607047F2
:1036A000843B002000300040034B1A681AB9034ADB
:1036B000D2F874281A607047803B00200030024026
:1036C000024B4FF08072C3F87428704700300240FC
:1036D00008B5FFF7E9FF024B1868C0F3407008BD5A
:1036E000803B002008B5FFF7DFFF024B1868C0F3EE
:1036F000007008BD803B0020EFF3098305494A6B49
:1037000022F001024A63683383F30988002383F3BC
:103710001188704700EF00E0202080F3118862B626
:103720000C4B0D4AD96821F4E0610904090C0A43E5
:10373000DA60D3F8FC20094942F08072C3F8FC201B
:103740000A6842F001020A601022DA7783F8220048
:10375000704700BF00ED00E00003FA05001000E034
:1037600010B5202383F311880E4B5B6813F40063BC
:1037700014D0F1EE103AEFF30984683C4FF08073F7
:10378000E361094BDB6B236684F30988FFF7FEFBDB
:1037900010B1064BA36110BD054BFBE783F3118805
:1037A000F9E700BF00ED00E000EF00E03B06000895
:1037B0003E06000870470000FEE700000A4B0B4879
:1037C0000B4A90420BD30B4BDA1C121AC11E22F08B
:1037D00003028B4238BF00220021FDF74BBE53F895
:1037E000041B40F8041BECE714400008083C0020D0
:1037F000083C0020083C00207047000000F080B822
:103800004FF08043002258631A610222DA60704749
:103810004FF080430022DA60704700004FF0804391
:10382000586370474FF08043586A70474B68436055
:103830008B688360CB68C3600B6943614B6903622B
:103840008B6943620B6803607047000008B5234B27
:1038500023481A6942F0FF021A611A6922F0FF0236
:103860001A611A691A6B42F0FF021A631A6D42F06C
:10387000FF021A651B4A1B6D1146FFF7D7FF02F1C5
:103880001C0100F58060FFF7D1FF02F1380100F55F
:103890008060FFF7CBFF02F1540100F58060FFF775
:1038A000C5FF02F1700100F58060FFF7BFFF02F174
:1038B0008C0100F58060FFF7B9FF02F1A80100F567
:1038C0008060FFF7B3FF02F1C40100F58060FFF7ED
:1038D000ADFFBDE8084000F097B800BF00380240D7
:1038E00000000240043F000808B500F017FAFFF797
:1038F0007BFBBDE80840FFF7D7BE00007047000023
:10390000104B1A6C42F001021A641A6E42F0010266
:103910001A660D4A1B6E936843F0010393604FF0E3
:10392000804331229A624FF0FF32DA6200229A61BC
:103930005A63DA605A6001225A6108211A601C2019
:10394000FFF744B800380240002004E04FF0804206
:1039500008B51169D3680B40D9B2C9439B071161FF
:1039600007D5202383F31188FFF75EFB002383F341
:10397000118808BD08B5FFF7E9FFBDE80840FFF76B
:10398000EFBE00001E4B1A6962F0FF021A611A694D
:10399000D2B21A614FF0FF301A695A69586100219A
:1039A0005A6959615A691A6A62F080521A621A6A2F
:1039B00002F080521A621A6A5A6A58625A6A596246
:1039C0005A6A1A6C42F080521A641A6E42F080529F
:1039D0001A661A6E0B4A106840F480701060186FF7
:1039E00000F44070B0F5007F1EBF4FF480301867C0
:1039F0001967536823F40073536000F06FB900BF78
:103A000000380240007000403B4B3C4A1A643C4A7C
:103A10004FF4404111601A6842F001021A601A68BE
:103A20009007FCD59A6822F003029A60324B9A689C
:103A300012F00C02FBD1196801F0F90119609A60CB
:103A40001A6842F480321A601A689103FCD55A6FE2
:103A500042F001025A67284B5A6F9207FCD5294A57
:103A60005A601A6842F080721A60254A53685804F6
:103A7000FCD5214B1A689101FCD5234AC3F8842058
:103A80001A6842F080621A601A681201FCD51F4A57
:103A90009A600322C3F88C204FF00062C3F8942090
:103AA0001B4B1A681B4B9A421B4B21D11B4A1168B6
:103AB0001B4A91421CD140F203121A60164A136845
:103AC00003F00F03032BFAD10B4B9A6842F002026A
:103AD0009A609A6802F00C02082AFAD15A6C42F4F1
:103AE00080425A645A6E42F480425A665B6E704756
:103AF00040F20372E1E700BF00380240000400100A
:103B000000700040081940021030002400948838EA
:103B1000002004E011640020003C024000ED00E0C1
:103B200041C20F41084A08B5516913680B4003F0C0
:103B30000103536123B1054A13680BB150689847DC
:103B4000BDE80840FFF70CBE003C0140883B002068
:103B5000084A08B5516913680B4003F0020353612A
:103B600023B1054A93680BB1D0689847BDE8084077
:103B7000FFF7F6BD003C0140883B0020084A08B52D
:103B8000516913680B4003F00403536123B1054AE4
:103B900013690BB150699847BDE80840FFF7E0BDD5
:103BA000003C0140883B0020084A08B55169136871
:103BB0000B4003F00803536123B1054A93690BB12D
:103BC000D0699847BDE80840FFF7CABD003C0140F6
:103BD000883B0020084A08B5516913680B4003F080
:103BE0001003536123B1054A136A0BB1506A984719
:103BF000BDE80840FFF7B4BD003C0140883B002011
:103C0000174B10B55A691C68144004F478725A6155
:103C1000A30604D5134A936A0BB1D06A984760068D
:103C200004D5104A136B0BB1506B9847210604D58D
:103C30000C4A936B0BB1D06B9847E20504D5094A47
:103C4000136C0BB1506C9847A30504D5054A936CCF
:103C50000BB1D06C9847BDE81040FFF781BD00BFA5
:103C6000003C0140883B00201A4B10B55A691C6883
:103C7000144004F47C425A61620504D5164A136D5F
:103C80000BB1506D9847230504D5134A936D0BB1C2
:103C9000D06D9847E00404D50F4A136E0BB1506EF7
:103CA0009847A10404D50C4A936E0BB1D06E984787
:103CB000620404D5084A136F0BB1506F9847230470
:103CC00004D5054A936F0BB1D06F9847BDE81040FB
:103CD000FFF746BD003C0140883B0020062108B5A7
:103CE0000846FEF773FE06210720FEF76FFE062149
:103CF0000820FEF76BFE06210920FEF767FE06216D
:103D00000A20FEF763FE06211720FEF75FFEBDE8DE
:103D1000084006212820FEF759BE000008B5FFF72D
:103D200031FE00F00BF8FEF767FEFFF767F8FFF7CC
:103D3000E5FDBDE80840FFF761BD00000023054A2E
:103D400019460133102BC2E9001102F10802F8D123
:103D5000704700BF883B002010B5013902449042F3
:103D600001D1002005E0037811F8014FA34201D0F2
:103D7000181B10BD0130F2E72DE9F041A3B1C91ABB
:103D800017780144044603F1FF3C8C42204601D9D8
:103D9000002009E00578BD4204F10104F5D10CEBE7
:103DA0000405D618A54201D1BDE8F08115F8018DB2
:103DB00016F801EDF045F5D0E7E70000034611F8ED
:103DC000012B03F8012B002AF9D170476F72672E7F
:103DD0006172647570696C6F742E5369657272617B
:103DE0002D463950000000004E6F20617070207326
:103DF00069670A00426164206677206C656E6774AB
:103E0000682025750A0042616420626F6172645FF8
:103E100069642025752073686F756C642062652065
:103E200025750A00426164206677206465736372B9
:103E30006970746F72206C656E6774682025750AEE
:103E40000042616420617070204352432030782525
:103E50003038783A30782530387820307825303846
:103E6000783A3078253038780A00476F6F642066DA
:103E700069726D776172650A0040A2E4F16468912D
:103E80000600000000000000C52D0008B12D00084C
:103E9000ED2D0008D92D0008E52D0008D12D0008D2
:103EA000BD2D0008A92D0008F92D00086D61696E6F
:103EB0000000000069646C6500000000B43E00086A
:103EC000C0390020383B002001000000E52F000829
:103ED0000000000000400000004000000040000022
:103EE000004000000000010000000200000002008D
:103EF00000000200000002000000020000000200BA
:103F000000000200A000282800000000AAAAAAAA17
:103F100050001424FFFF000000770000700700002D
:103F200001000A0000000000AAAAAAAA00000000DE
:103F3000FFFF0000000000008800000014000001E6
:103F400000000000A6AAAAAA00000001F9FF0000D4
:103F50000000000000000000000000000000000061
:103F6000AAAAAAAA00000000FFFF000000000000AB
:103F7000000000000000000000000000AAAAAAAA99
:103F800000000000FFFF0000000000000000000033
:103F90000000000000000000AAAAAAAA0000000079
:103FA000FFFF000000000000000000000000000013
:103FB00000000000AAAAAAAA00000000FFFF00005B
:103FC00000000000000000000000000000000000F1
:103FD0000A000000000000000300000000000000D4
:103FE000000000002CC2FF7F010000000000000064
:103FF0000A0400000000000000000F0000000000A4
:10400000640000000000000040420F00FE2A010092
:04401000D2040000D6
:00000001FF
